:020000020000FC
:1000000081CE00000000000020C0BCC18EC00000F6
:10001000000098C000000000000000000203040679
:10002000080C10182030406080000406080C1018DE
:100030002030406080A0C0000003070F1F000D0D9E
:100040000403060D0503030202004FB662FD0CC057
:10005000552041F00994C52DC095089483FDC7959E
:10006000C4BD64604FBE1895C0916400089483FDC0
:10007000C795C4BD6B7FC0916400CF3F09F41EC01B
:1000800070FF1AC082FD05C04FBE93989498959852
:10009000189576FD0EC065FD0CC0C091B100C0FD85
:1000A0009298C1FDC298C2FDC198CAEFC095CA9589
:1000B000F1F79398949895984FBE189524BCCC2747
:1000C000C064C8BF6460F8CFC6CF70FFC4CF65FD01
:1000D000C2CF939AC0CF70FFBECF65FDBCCF949ABC
:1000E000BACF70FFB8CF65FDB6CF959AB4CF929ACC
:1000F00070FFB1CF65FDAFCFC7E0CA95F1F7939A16
:10010000AACFC29A70FFA7CF65FDA5CFC7E0CA9559
:10011000F1F7949AA0CFC19A70FF9DCF65FD9BCF58
:10012000C7E0CA95F1F7959A96CF4FB6C9B7CF7E7B
:10013000C9BF6E7FCCB5CE0DDDB5DF1DDBBDCABD41
:100140004FBE18953FB68F7EA9B7A072A2118061ED
:10015000A9B7AF7DA9BFA9B7AE7FA9BF7894A09179
:100160006800AA2341F085FD2BC0A0916800AA95E4
:10017000A093680025C040E050E085FD15C0A6B3FF
:1001800096FDA095A0FD4FEFAEB5A06496FDAF7BA8
:10019000AEBDAA27A062A8BF8D7FA6B396FDA0958D
:1001A000A0FD5FEF451739F7A0E461FDA09368005B
:1001B00085FD03C0A0E4A093680040939600816091
:1001C00085FD0EC0A0916900AA2331F0A0916900BD
:1001D000AA95A093690004C08061AA27A062A8BF65
:1001E00080FF0AC0A09196004A2F61FF8E7F85FD97
:1001F00001C000C0409361004091B400443009F058
:1002000004C0A0916100A0936300A52DA03408F064
:100210006860A0916000A395A093600059F0F894E5
:10022000A9B7A160A9BF84FF03C0A9B7A062A9BFF5
:100230003FBE1895A0917400A395A093740042E06E
:1002400050916800552329F085FF03C05A955093BB
:100250006800A0919600A13018F0209299000DC07E
:1002600020929A002092A300A0919900AF5FA093E2
:10027000990018F0AFEFA0939900B09061005091F1
:10028000B400523049F466FF91F0A2E3BA1678F058
:10029000A0918600A0936100533049F466FF39F0C5
:1002A000A2E3BA1620F0A091C000A0936100509183
:1002B00062005B1521F010F05A9501C053955093E0
:1002C00062004A95D1F65091A300539509F45A95CE
:1002D0005093A300A091A400AA95A093A40009F0B4
:1002E00046C0A1E0A093A40045E0A091A5005A1744
:1002F000F0F1A091A6005A1728F441E0A3E0A093E2
:10030000A40007C0A091A7005A1718F441E0409339
:10031000A400D0909C00C0906300DC14A8F0A091D1
:10032000B400A430D9F066FD0FC0C0929C00539574
:1003300011F0A091A500A093A300A1E0A093A400B8
:10034000ACE3A093620013C0A0919C00A40F20F422
:100350005FEF50939C0002C0A0939C00A0919C0072
:10036000AF3F29F4AFEFA0939A00A093A300F894B5
:10037000A9B7A160A9BF84FF03C0A9B7A062A9BFA4
:100380003FBE18953FB646B557B58F7EA9B7A07248
:10039000A2118061A9B7AF7DA9BFA9B7AE7FA9BFE0
:1003A000789481FD25C0AEB5AF7B96FDA064AEBD4F
:1003B0008260A6B396FDA095A0FF05C0409365009E
:1003C000509366001FC1AEB5A06496FDAF7BAEBD75
:1003D000AA27A062A8BF8D7F85FF01C006C140E0AB
:1003E000A6B396FDA095A0FD00C140939600EFC076
:1003F000AEB5A06496FDAF7BAEBD8D7F61FF72C0D0
:10040000AEB5AF7B96FDA064AEBDAA27A062A8BF23
:1004100082604093910050939200A0908F004A19FF
:10042000B09090005B09BB24A22C4C38520518F404
:100430002092950049C0A091D400AA2359F1483CCC
:10044000520528F4A0E1BA2EAAE0AA2E23C048360D
:10045000A1E05A0728F4A8E0BA2EAFE0AA2E1AC0ED
:10046000403DA2E05A0728F4A4E0BA2EAEE1AA2E3D
:1004700011C0403AA5E05A0728F4A2E0BA2EACE336
:10048000AA2E08C04839A8E05A0720F4A1E0BA2EE5
:10049000A8E7AA2EC42EA0919300CA1AD52EA09127
:1004A0009400DA0ADD202AF4AFEFC094D094CA1A7F
:1004B000DA0A20929500A8E0A210A0E0CA14DA0699
:1004C00018F4A1E0A09395004093930050939400FA
:1004D000409191005091920040938F005093900072
:1004E00042E075C0A09165004A1BA09166005A0BBE
:1004F00094FD60C093FD5EC092FD5AC086FF03C0AC
:10050000D52EC42E0CC05695479591FD51C05695D9
:10051000479590FD4DC0D52EC42ED694C79461FD4D
:1005200019C0AC2DAC51AD2DA24008F005C0DD20A6
:1005300089F4AC2DA85C70F4A0916700A395AA2360
:1005400011F0A0936700AA3008F44FC020929600E3
:1005500081604BC0A0916700AA2319F0AA95A093CF
:100560006700A22C5091BA0097FD02C0A090C8006D
:10057000AAEFAA0EA22DA21DCA18DA0A4FB741701F
:10058000442319F040E050E015C0AFEFCA16D20482
:1005900018F04FEF50E00EC0A091AC00CA9E412D64
:1005A000000C441F50E008F012C04FEF50E00FC0A5
:1005B0005695479594FF07C0552309F04FEFA42F98
:1005C000A6954A0F521D4F3F520508F04FEF40933A
:1005D0009600816061FF09C0AFE1A095A923AB2916
:1005E0009A2F8F7DBB2009F48062A0E4A09368005D
:1005F00085FF03C0AAE0A093680061FD03C085FDEC
:1006000001C08F7E85FD03C0A0E2A0936900F8942D
:10061000A9B7A160A9BF84FF03C0A9B7A062A9BF01
:100620003FBE189511E00AC013E008C01AE006C0EA
:100630001EE104C014E602C018EC00C005E1BB27AF
:10064000BA95F1F70A95D9F71A95C1F708952AE3F3
:1006500038E709C020E33CE806C02AE234EB03C0D7
:1006600025E238EC00C012E0BB27C29ABA95F1F738
:10067000949ABA95F1F79498BA95F1F7C298BA9509
:10068000F1F7123009F0939A123009F4959AB0916B
:10069000AD00BA95F1F7123009F09398123009F4D1
:1006A0009598B7E8BA95F1F71A95F1F6022FB22F9F
:1006B000BA95F1F70A95D9F73A95A9F6C29A08952D
:1006C000221B39E0001F3A9509F40895221F211BCF
:1006D00018F4210F8894F6CF0894F4CF622C722C72
:1006E000B0E08894B395221F331FE0F73795279524
:1006F0008894912E802E020B130B10F4192D082DC7
:1007000010F4889401C00894661C771CBA9571F7A0
:10071000172D062D0895322D11232AF43A950095B0
:100720001095031B130BF894029F712C002D129F40
:10073000912C802C7894780C172D921C292DB4E0E4
:100740006B2E2695179507956A94D9F7332321F0D8
:1007500000951095031B130B08950091B40004300D
:1007600009F474C0B0919600B95198F0B72FB670E3
:1007700081F466FD2BC005E09090C600B92DBA95B6
:1007800021F00AE0BA9509F002E1B0917B00B01BBC
:10079000E0F066FF0AC0B0919E00B0939C00BFEFEE
:1007A000B093A300B1E0B093A400B0916100B09306
:1007B000630020927E0020927F0020928000209291
:1007C0008100209282006F7B41C060649090C600DF
:1007D000B92DBA9579F4B0916200B095BB1FBB1FDB
:1007E0001B2FB7950B2FB12FB170B3951B2FB02FC7
:1007F000BE7F25C0B92DBA95BA9581F4B09162003B
:10080000B095BB1FBB1FBB1F1B2FB7950B2FB12F65
:10081000B370B3951B2FB02FBC7F14C0B091620092
:10082000B095BB1FBB1FBB1FBB1F1B2FB7950B2F4B
:10083000B12FB770B395B3951B2FB02FB87FB054BD
:100840000B2F120900937E0010937F0008951091E2
:100850007B00169500917A000795B0917E00B01B41
:100860000B2FB0917F00B10B1B2F28F40038BFEF86
:100870001B0740F009C00F37120508F405C00FE749
:1008800010E002C000E81FEF009383001093840083
:10089000089500918300B09180000B0F10918400A7
:1008A000B09181001B1F20E03091840033230AF4B3
:1008B0002A95B09182002B1F1AF4203F40F00AC005
:1008C0002F3008F407C00FEF1FEF2FE003C000E048
:1008D00010E020EF30916300B0919B003B1718F4BB
:1008E000323030F009C0B0918400BB235AF004C00C
:1008F000B0918400BB2332F40093800010938100F8
:100900002093820008952091D70000918300000F6A
:1009100010918400111FFFDE11232AF40038BFEF6D
:100920001B0740F009C00F37120508F405C00FE798
:1009300010E002C000E81FEF002352F0B091620007
:10094000B01B0B2F18F0013008F00AC001E008C0FE
:1009500000950F5FB09162000B0F08F001C00FEF20
:100960000093850008952091D80000918100109196
:100970008200D1DE11232AF40130BFEF1B0740F0C3
:1009800009C00F3F120508F405C00FEF10E002C0C8
:1009900001E01FEF112352F0B0918500B01B0B2F27
:1009A00018F0013008F00AC001E008C000950F5FA0
:1009B000B09185000B0F08F001C00FEF00936300AA
:1009C00008950FEF677F71FD29C072FD09C068604F
:1009D000B0917B00BA3020F0B52DB03408F4677FB9
:1009E000B091D300BB23D1F0B0917B00BB23B1F019
:1009F0000FEF10917B0064DEF894B091730072FDEC
:100A0000B5E00B9F112D002D7894112309F00FEF05
:100A1000B0919E000B1710F400919E0000939D0072
:100A2000089500917A0010917B0000541140B0911C
:100A30009D0010F4BA9501C0B39511F0B0939D00DC
:100A40000895F3D3B7E074FDB6E0B06CB7B9B6B1B2
:100A5000B068B064B6B9E6DDB7E074FDB6E0B06C7E
:100A6000B7B9B6B1B068B064B6B9B6B1B6FDFDCF2E
:100A700004B115B1B6B1BF77B6B930D42AEB209323
:100A8000A800222309F441C030E03093A900732E5E
:100A90007694622E6694620E731E262D372D0217F1
:100AA000130778F08090A800BAEBB80DB093A800B7
:100AB0008090A900B0E0B81DB093A900260D371DA5
:100AC000EECF8090A8009090A9001091A9001695F3
:100AD0000091A80007951695079523E016950795B0
:100AE0002A95E1F72091B5002A9529F42092A800D3
:100AF0002092A9000AC02A9521F0800E911E2A9505
:100B0000E1F78092A8009092A90008952091B50085
:100B1000B6B1B6FDFBCF04B115B1B6B1BF77B6B96A
:100B2000B091AA00B395B093AA00B83060F12092BA
:100B3000AA00B091D200BB2321F1112329F0B0917A
:100B4000AB00BF3F61F009C0B091AB000B1739F0AB
:100B500020F4BB2321F0BA9502C0B395E1F30091D4
:100B60009B00B093AB00B93B50F400ECBA3A38F4B8
:100B700000E8BB3920F400E4BC3808F400E000933E
:100B80009B007F7E08952130B1F00F3FB3E01B073B
:100B900090F4BAEBBB2379F0B091A8000B17B09199
:100BA000A9001B0740F4B0919B00BB2359F0BA95F4
:100BB000B0939B0007C0B0919B00BF3F19F0B39565
:100BC000B0939B0000919B00B0916300B01B10F4A8
:100BD00000916300B0919C000B1750F000919C00B5
:100BE000B0919C00BF3F21F0B0919C00B0939B005E
:100BF000502E00936400B091AA00B73009F47061E0
:100C0000089502E3F894B091D9000B9F012D000CD8
:100C1000001F7894B0919B000B1710F000919B007F
:100C20000093610000936300502E009364000093D2
:100C30009E00089520927A00B0EFB0937B00089553
:100C4000F8940CB51DB5209174007894309175001E
:100C5000609076000093750010937600031B1609D0
:100C600071FD03C077FD7DC027C070907700209391
:100C700077002709222311F00FEF1FEF80907800F3
:100C8000909079003093780060927900009175001F
:100C9000109176000819190920917A0030917B0093
:100CA00036952795020F131F10F40FEF1FEF0093D7
:100CB0007A0010937B0029C020917A0030917B004C
:100CC0003901B4E08B2EB2E09B2E343010F08A94C0
:100CD0009A94383010F08A949A94769467948A940F
:100CE000E1F726193709992021F0169507959A946E
:100CF000E1F7200F311F20937A0030937B0028F416
:100D00003FEF30937A0030937B00323008F4706804
:100D100071FF02C0B3E00DC0B091C400009171003A
:100D2000023838F0B395003A08F0B395B63008F0C1
:100D3000B5E09B2EB4E08B2E10917B0000917A00E1
:100D400024E0169507952A95E1F70819120928F06D
:100D5000B02FB250B12FB20910F402E010E09801A8
:100D600026C020917A0030917B00390176946794F7
:100D70006694669466942619320906950695200FA6
:100D8000321D20937A0030937B00323008F07F7759
:100D900004E0369527953695279526952695201BB0
:100DA00010F0223008F422E089019090C40060FD28
:100DB000FECFE0908B00F0908C006160B9B7B0611D
:100DC000B9BF380177FD41C07694679400938B00DA
:100DD00010938C00B92DB330E1F0B0FD04C0060DC6
:100DE000171D930106C0000F111F0250120922E0C7
:100DF00030E0B92DB33068F020938D0030938E0031
:100E000000938700109388006092890070928A0096
:100E10003AC000938D0010938E002093870030938A
:100E200088006092890070928A0071FF0DC0BFE057
:100E3000B0938D0020928E00B093890020928A009A
:100E4000B0938B0020928C001EC0669400938B00A0
:100E5000B92DB33091F0B0FD03C0060D262D03C0AF
:100E6000000F025022E0B92DB33038F020938D00EE
:100E7000009387006092890006C000938D00209344
:100E800087006092890000917C0002FD03500130D0
:100E900049F495FD12C0B0B7B860B0BFB0E0B06C17
:100EA000B7B90EC0023039F4B0B7B860B0BFB1E026
:100EB000B06CB7B905C095FDEECFB0B7B77FB0BF86
:100EC0000091A200000F10F4BBE60B270093A200D4
:100ED00060FDFECFB2E0B0936E006160B9B7B06163
:100EE000B9BFB72FB670D1F020917A0030917B0056
:100EF000369527953695279571FF02C0B0E43B0FD4
:100F0000F8940CB51DB5020F131F1BBD0ABD61601F
:100F1000B0E1B8BFB9B7B061B9BF78940895606166
:100F200020927D0020E067FD20E206C060612092F3
:100F30007D0020E267FD20E001E011E077FD11C0B7
:100F4000B72FB67009F06F7E14E100917B00069513
:100F500009F403950F3008F00FE071FF02C004E1BF
:100F600014E160FD0FC0B0917D00BB2359F071FF0B
:100F700006C0B0916E00BA95B0936E0011F4706225
:100F800049C0ABDFB0B73B2FB77FB0BFB8B1B0B788
:100F900033FDB860B0BFB0917D00B395B0937D00D4
:100FA000B8B177FD06C0B1E071FDB3E0BA95F1F7D5
:100FB000B8B1B072B21709F022C071FF05C0039535
:100FC000011708F00A95CDCF64FD05C00395011700
:100FD00008F0B2CFC6CF6F7EF8943CB56DB4709078
:100FE0007A0080907B00370D681C6BBC3ABD616055
:100FF000B0E1B8BFB9B7B061B9BF78949DCFB09137
:101000006D00B13008F498CF64FD96CF0A9509F0D1
:10101000A8CF7F7D20918D0030918E00F894B0E1B3
:10102000B8BF0CB51DB5020F131F1BBD0ABDE09064
:101030008700F09088006160B9B7B061B9BF78945B
:10104000B72FB67039F0B0916D0072FFB395B093C1
:101050006D0009C075FF07C067FD05C064FD03C0D2
:10106000BF91BF91F6C4089500E063FF03C064FF21
:1010700001C001E0F89410917100B7E01B9F212D91
:10108000102D7894200F269517952695179526955F
:10109000179510937100183718F4B8E7B0937100E2
:1010A00000917100B09172000B1720F0606293986C
:1010B0009498959860FDFECFE0908900F0908A00AA
:1010C0006160B9B7B061B9BF0895AC98B2E095FD61
:1010D0000AC0F894B0937C00C29A929862FF01C053
:1010E000959A7894F9C0F894B0937C00C29AC1980C
:1010F00062FF01C0939A7894EFC0AC9AB3E082FF8C
:1011000024C095FD11C002E0F894B0937C00E1E8A2
:10111000F0E00093B1009598C19A62FF02C0949AE2
:1011200001C0C2987894D8C002E0F894B0937C00D3
:10113000E1E8F0E00093B1009398929A62FF02C058
:10114000949A01C0C2987894C7C095FD0BC0F894DA
:10115000B0937C00EBE6F0E0959862FF01C0949AB2
:101160007894BAC0F894B0937C00EBE6F0E09398E2
:1011700062FF01C0949A7894AFC0AC98B4E095FD3A
:101180000AC0F894B0937C00929AC19862FF01C0A3
:10119000949A7894A1C0F894B0937C00C19A9298E4
:1011A00062FF01C0949A789497C0AC9AB5E082FF30
:1011B00024C095FD11C001E0F894B0937C00E7E7EE
:1011C000F0E00093B1009498C29A62FF02C0939A33
:1011D00001C09298789480C004E0F894B0937C00A9
:1011E000EBE8F0E00093B1009498C29A62FF02C06D
:1011F000959A01C0C19878946FC095FD0BC0F89482
:10120000B0937C00E5E6F0E0949862FF01C0939A09
:10121000789462C0F894B0937C00E1E7F0E0949891
:1012200062FF01C0959A789457C0AC98B6E095FDDE
:101230000AC0F894B0937C00C19AC29862FF01C0C2
:10124000939A789449C0F894B0937C00929AC2988B
:1012500062FF01C0959A78943FC0AC9AB1E082FFDA
:1012600024C095FD11C004E0F894B0937C00EBE835
:10127000F0E00093B1009398929A62FF02C0959AB1
:1012800001C0C198789428C001E0F894B0937C0024
:10129000E7E7F0E00093B1009598C19A62FF02C0C1
:1012A000939A01C09298789417C095FD0BC0F8945A
:1012B000B0937C00E1E7F0E0939862FF01C0959A5B
:1012C00078940AC0F894B0937C00E5E6F0E0959835
:1012D00062FF01C0939A78946F7D089524E630E010
:1012E000F9012092B100939894989598929AC29A95
:1012F000C19A6B7F0895A2EBB0E007E00D9307E081
:101300000D9301E00D9304E00D930FEF0D930D93FA
:1013100009E00D9302E00D9301E00D9301E00D93C0
:10132000AEEBB0E001E00D9300E00D9304EB0D9304
:101330000FEF0D930D930D9303E00D930FEF0D93AE
:1013400001E00D930FEF0D9305E20D9300ED0D936A
:1013500008E70D9308EC0D9304E00D930FEF0D9348
:1013600001E00D9300E00D930AE70D930AE00D9361
:1013700000E00D9301E00D9300E00D930FEF0D934E
:1013800000E00D9308952091B9008B7F233009F47C
:101390008460B091BA009F7DB1FD90629F7BB09157
:1013A000BB00B1FD9064223011F0886001C0877FDE
:1013B00008950A95E00FF21DB4910895ECE1F0E074
:1013C0000091B200F6DFB093D700ECE1F0E00091BD
:1013D000B300EFDFB093D800EAE2F0E00091B8008C
:1013E000E8DFB093D9000091D100002309F4039500
:1013F000013108F001E1B02FB00FB00FB093A5009C
:101400001B2FB10FB10FB00FB093A600B10FB00FEB
:10141000B00FB093A7000091B800023008F402E0CA
:1014200000937300B091CE000FEFB23009F400EAE0
:10143000B33009F402E800937200E8E3F0E00091B1
:10144000D500B7DFB093A000089508952091C8009B
:101450003091C900B091BA00B33009F43E5097FF03
:1014600002C020E03FEFB32FB21B6B2EB25810F436
:10147000B2E86B2E00E00395609EB12DBD57D8F306
:101480000093AC0008959068E1DFD2D820E030E00E
:10149000B0E16B2EC9D8B09196002B0F321D6A9423
:1014A000C9F7B4E036952795BA95E1F7822E9F7774
:1014B000CDDF0895F894E3E0F0E0B9E0B7BFB49170
:1014C000B078C1F3F894A895B1B5B861B1BDB0E0FA
:1014D000B1BDB4E0BEBFBFE5BDBF00DFB6E0B8BB85
:1014E000B6E1B7BBB8E0B5BBBCE1B4BBB4E0B2BBDE
:1014F000BCE3B1BB2224A0E0B0E02D92AA31E9F711
:10150000A0E6B0E00FEF2D920A95E9F7B1E0B093B5
:10151000A200F1DEDFD2B7E0B06CB7B9B6B1B4600B
:10152000B068B6B90091CA000093AD00B1E0B093C5
:101530006A00F89481D88BD87BD88CD879D88DD88C
:1015400077D857D379D878D875D8F8940AEF1AEFA6
:10155000A6B396FDA095A0FF1FC01A95C9F70A95DE
:10156000B1F7E0E0FCE1B591B43E39F4B591B03E9D
:1015700021F4B591BF3F09F40CC0E0E0F395F39579
:10158000B591B83F49F4B591B43931F4B591BA3A4F
:1015900019F4EE27F6950994F6DE10DF56DF56DFD4
:1015A0000091CA000093AD0099DEB2E0B3BFB2E093
:1015B000BEBDB2E0B5BDB1E5B8BFB9BFB0B70B2F86
:1015C000B77FB0BFB8B1B0B703FDB860B0BF2AD81D
:1015D000789437DA20927000BEB5B06496FDBF7B78
:1015E000BEBDB9B7B062B9BFBB27B062B8BF8D7F0F
:1015F00023D8626033E02CE0B0919500BB2321F446
:101600002CE03A9509F4A1CF13D880FF9ECF8E7FAE
:10161000B0919600B23078F3B92FBF710091980065
:1016200000939700B0939800B01729F72A9521F7F7
:101630006D7FBEB5B06496FDBF7BBEBDBB27B062FB
:10164000B8BF8D7FB091D400BB2321F48062B92F45
:10165000B0709B2F8F7B20926700ECD785FF05C071
:10166000B0916700BA3008F08064DED702E085FFF1
:1016700001C000E0B0919600B017B8F3F894E7D736
:10168000E6D7E5D77894D8D720928600CDD7B09109
:10169000BE00B13008F46EC0B0916A00B13008F4F9
:1016A00069C085FD18C0B0919600BF3F08F462C0C4
:1016B000F894D6D77894BED7B0919600B130C0F7E1
:1016C000F894C5D7B3D7C3D77894B4D7B091960060
:1016D000BF3FB0F3C0C2B8E09B2E9068F894B6DE6E
:1016E0007894A8D7F8949F77B1DE80909600B09157
:1016F0009600BF37789408F445C094D7F894B0D7D3
:1017000078949A9451F7BFDEB82DB550B093C900C4
:1017100093D7F8940CD272D27894BAE09B2E90684A
:10172000F89494DE789486D7F8949F778FDE809033
:101730009600B0919600BF37789478F773D7F894F5
:1017400086D774D784D778949A9449F79CDEB82DBD
:10175000BB5FB093C80070D7F894E9D15ED278949B
:1017600069D7F89473DE7894B0919600BF3F08F47F
:1017700098CF71C200919600B09186000B1710F0BF
:101780000093860057D701E0B091BA00B35009F436
:1017900005E0B0919600B01708F078CFF89460D7C4
:1017A0005FD75ED7789448D720926A0020926B006A
:1017B00020926C00B0916B00B395B0936B00BF3F6B
:1017C00071F5B0916C00B395B0936C00B091CC0002
:1017D00009E1BA9559F002E3BA9541F00DE7BA95DF
:1017E00029F00AEFBA9511F020926C00B0916C00CC
:1017F000B017A8F073DD16D7B0916C00BA95B0930E
:101800006C0020926B00B091CB00B093AD00F894C7
:1018100027D77894B091CA00B093AD000BD706D704
:10182000B0916800BB2319F485FF01C08ECE01E0A2
:1018300085FD01C006E0B0919600B01708F4BACF5C
:10184000F9D6B0916800BB2309F47FCEF89446DD49
:10185000209261002092620020926300522C20921C
:1018600064002092A1007894B091B700BB0FB093B0
:101870009F0020927E0020927F0020928000209284
:101880008100209282002092AA0060E070E0209205
:101890007100B8E0B093AA007061C4D6B7E074FDDF
:1018A000B6E0B06CB7B9B6B1B068B064B6B9B6B1AD
:1018B000B6FDFDCF04B115B1B6B1BF77B6B91123EE
:1018C00009F00FEF0093AB0021D9B8E0B093AA0064
:1018D000706159DDF894BFEFB0939B0092D9B0913D
:1018E0006100B0939B00B0939C00B0939D007894EE
:1018F000B1E0B0936100B09363005B2EB0936400DD
:10190000B093A400B0919A00B093A300B091BA0034
:10191000B33019F49F7D87FD9062716072602092F0
:101920006D0083DC9ADC86D98BD984D989D982D998
:10193000FDDA13D799DBC9DB83D9F1DA66FD87D7E6
:1019400077FF3FD877FD6DD88FDBD7DB79D9EEDA1B
:1019500066FD9FD789DB11DC73D9E1DA66FDD3D749
:1019600083DB23DC6DD9E2DA66FDFDD77DDB5DDC50
:1019700067D9D5DAB7E074FDB6E0B06CB7B9B6B1E7
:10198000B068B064B6B970DB68DC5AD9BFD871FFF3
:101990001EC0B0919E00B0939B00B0939C00B0918C
:1019A0009A00B093A300B1E0B093A40018E12CE03A
:1019B000B0916D00B11728F07D7F746020936F00A7
:1019C00006C0B0919600B13008F0B2CF4CC072FFA3
:1019D00011C067FD0FC0B0916F00BA9519F47B7FFD
:1019E0007860A6CFB0936F00B0919600B13008F048
:1019F0009FCF39C020927000B0919900B13058F05B
:101A0000B0919E00B0939C00B0919A00B093A30057
:101A1000B1E0B093A400B09199000AEF1091D60004
:101A2000112309F003E0B01708F01DC085FF04C0C2
:101A3000B0916800BB23B9F000EF67FF05C0B0911B
:101A40009E00B0939B0000E2B0917B00B01708F4B9
:101A50006FCFB0917000B395B0937000B0919600C5
:101A6000BB2309F002C020927000F89437DC80900C
:101A7000B900B2E0B093B90086DC8092B900209240
:101A800061002092620020926300522C2092640038
:101A900020929F0060E070E07894CCD51FDC00912C
:101AA000D600002319F0939A949A959AB7E0B06CF7
:101AB000B7B9B6B1B460B068B6B985FF05C0B0912A
:101AC0006800BB2309F441CDB091BF00B13008F0EC
:101AD000CCCD6CCEEDE0F0E023D0053A09F01BC090
:101AE000EEE0F0E01DD00A3509F015C03AE0A2EBB7
:101AF000B0E0E3E0F0E014D00D9331963A95D9F7D9
:101B000039E1AEEBB0E0EFE0F0E00AD00D933196B2
:101B10003A95D9F702C0EFDB0AD0E8E2F0E0089589
:101B2000E199FECFEEBBFFBBE09A0DB308951ED046
:101B30003AE0A2EBB0E0E3E0F0E00D910FD0319697
:101B40003A95D9F739E1AEEBB0E0EFE0F0E00D9176
:101B500005D031963A95D9F712D00895E199FECF84
:101B60000DBBEEBBFFBBE29AE19A0895EDE0F0E019
:101B70000FEFF4DFEEE0F0E00FEFF0DF0895EDE0BF
:101B8000F0E005EAEBDFEEE0F0E00AE5E7DF0895DC
:101B90003091AE000091AF00313011F40093B200EB
:101BA000323011F40093B300333011F40093B400D9
:101BB000343011F40093C600353011F40093B500B1
:101BC000363011F40093B800373011F40093C4009C
:101BD000383011F40093B900393011F40093CE007D
:101BE0003A3011F40093BA003B3011F40093BB007B
:101BF000089525E021D52A95E9F7089528D52AD515
:101C00002CD52ED513D523D525D527D529D50ED519
:101C10001ED520D522D524D5089522D51ED51AD576
:101C200016D504D51DD519D515D511D5FFD418D580
:101C300014D510D50CD508958090AE009090AF00CB
:101C400006D505D504D5F2D48A94D1F709D5EED4BA
:101C50009A94E1F70895F894D1DF7894CADFC9DF48
:101C6000B1E0B093AE00B1E0B093AF002092B0000D
:101C7000F894E2DF7894B5E06B2E70909600DCD497
:101C8000B09196007B16C9F7B13018F0BF3F40F114
:101C900007C07EDFF8944BDFB1DFB8E0B1BDA9DF4C
:101CA0006A9459F7B091B000B395B093B000B330D7
:101CB00008F4DECF9EDFB091AF00B395B093AF00D4
:101CC000F894B091AE00BA95EEE3F0E0EB0FF21DA0
:101CD000049178940395B091AF00B01708F4C6CF83
:101CE00088DF87DFB091AE00B395B093AE00B091BE
:101CF000AE00BC3008F4B7CFFEDAF89418DFB8E0D5
:061D0000B1BD77DFD7CB77
:00000001FF
